 setfldw001

 Timestamp is 3a364a15 (reproducible build file hash)

 Preferred load address is 0000000180000000

 Start         Length     Name                   Class
 0001:00000000 00002d30H .text$mn                CODE
 0001:00002d30 00000036H .text$mn$00             CODE
 0001:00002d66 00000092H .text$x                 CODE
 0002:00000000 00000198H .idata$5                DATA
 0002:00000198 00000038H .00cfg                  DATA
 0002:000001d0 00000008H .CRT$XCA                DATA
 0002:000001d8 00000008H .CRT$XCZ                DATA
 0002:000001e0 00000008H .CRT$XIA                DATA
 0002:000001e8 00000008H .CRT$XIC                DATA
 0002:000001f0 00000008H .CRT$XIZ                DATA
 0002:000001f8 00000008H .CRT$XLA                DATA
 0002:00000200 00000008H .CRT$XLZ                DATA
 0002:00000208 00000008H .CRT$XPA                DATA
 0002:00000210 00000008H .CRT$XPZ                DATA
 0002:00000218 00000008H .CRT$XTA                DATA
 0002:00000220 00000010H .CRT$XTZ                DATA
 0002:00000228 00000000H .gehcont$y              DATA
 0002:00000228 00000000H .gfids$y                DATA
 0002:00000230 00001d50H .rdata                  DATA
 0002:00001f80 00000000H .rdata$CastGuardVftablesA DATA
 0002:00001f80 00000000H .rdata$CastGuardVftablesC DATA
 0002:00001f80 00000028H .rdata$T                DATA
 0002:00001fa8 000000b0H .rdata$voltmd           DATA
 0002:00002058 00000318H .rdata$zzzdbg           DATA
 0002:00002370 00000008H .rtc$IAA                DATA
 0002:00002378 00000008H .rtc$IZZ                DATA
 0002:00002380 00000008H .rtc$TAA                DATA
 0002:00002388 00000008H .rtc$TZZ                DATA
 0002:00002390 00000004H .tls                    DATA
 0002:00002394 00000004H .tls$                   DATA
 0002:00002398 00000008H .tls$ZZZ                DATA
 0002:000023a0 00000300H .xdata                  DATA
 0002:000026a0 00000464H .edata                  DATA
 0002:00002b04 00000064H .idata$2                DATA
 0002:00002b68 00000018H .idata$3                DATA
 0002:00002b80 00000198H .idata$4                DATA
 0002:00002d18 0000041eH .idata$6                DATA
 0003:00000000 00000170H .data                   DATA
 0003:00000170 0001b378H .bss                    DATA
 0004:00000000 00000390H .pdata                  DATA

  Address         Publics by Value              Rva+Base               Lib:Object

 0000:00000000       __AbsoluteZero             0000000000000000     <absolute>
 0000:00000000       ___safe_se_handler_count   0000000000000000     <absolute>
 0000:00000000       ___safe_se_handler_table   0000000000000000     <absolute>
 0000:00000000       __arm64x_extra_rfe_table   0000000000000000     <absolute>
 0000:00000000       __arm64x_extra_rfe_table_size 0000000000000000     <absolute>
 0000:00000000       __arm64x_native_entrypoint 0000000000000000     <absolute>
 0000:00000000       __arm64x_redirection_metadata 0000000000000000     <absolute>
 0000:00000000       __arm64x_redirection_metadata_count 0000000000000000     <absolute>
 0000:00000000       __dynamic_value_reloc_table 0000000000000000     <absolute>
 0000:00000000       __enclave_config           0000000000000000     <absolute>
 0000:00000000       __guard_check_icall_a64n_fptr 0000000000000000     <absolute>
 0000:00000000       __guard_eh_cont_count      0000000000000000     <absolute>
 0000:00000000       __guard_eh_cont_table      0000000000000000     <absolute>
 0000:00000000       __guard_fids_count         0000000000000000     <absolute>
 0000:00000000       __guard_fids_table         0000000000000000     <absolute>
 0000:00000000       __guard_iat_count          0000000000000000     <absolute>
 0000:00000000       __guard_iat_table          0000000000000000     <absolute>
 0000:00000000       __guard_longjmp_count      0000000000000000     <absolute>
 0000:00000000       __guard_longjmp_table      0000000000000000     <absolute>
 0000:00000000       __hybrid_auxiliary_iat     0000000000000000     <absolute>
 0000:00000000       __hybrid_auxiliary_iat_copy 0000000000000000     <absolute>
 0000:00000000       __hybrid_code_map          0000000000000000     <absolute>
 0000:00000000       __hybrid_code_map_count    0000000000000000     <absolute>
 0000:00000000       __x64_code_ranges_to_entry_points 0000000000000000     <absolute>
 0000:00000000       __x64_code_ranges_to_entry_points_count 0000000000000000     <absolute>
 0000:00000100       __guard_flags              0000000000000100     <absolute>
 0000:00000000       __ImageBase                0000000180000000     <linker-defined>
 0001:00000000       ?NewObject@JNIEnv_@@QEAAPEAV_jobject@@PEAV_jclass@@PEAU_jmethodID@@ZZ 0000000180001000 f i libsetfldw001.obj
 0001:00000024       ?SetEventNotificationMode@_jvmtiEnv@@QEAA?AW4jvmtiError@@W4jvmtiEventMode@@W4jvmtiEvent@@PEAV_jobject@@ZZ 0000000180001024 f i libsetfldw001.obj
 0001:0000002c       ?TranslateError@@YAPEBDW4jvmtiError@@@Z 000000018000102c f   libsetfldw001.obj
 0001:000002e4       ?nsk_jni_check_exception@@YAHPEAUJNIEnv_@@QEBDH@Z 00000001800012e4 f   libsetfldw001.obj
 0001:00000428       ?nsk_jni_lverify@@YAHHPEAUJNIEnv_@@HQEBDH1ZZ 0000000180001428 f   libsetfldw001.obj
 0001:000004c8       Agent_Initialize           00000001800014c8 f   libsetfldw001.obj
 0001:0000062c       Agent_OnAttach             000000018000162c f   libsetfldw001.obj
 0001:0000062c       Agent_OnLoad               000000018000162c f   libsetfldw001.obj
 0001:00000634       FieldAccess                0000000180001634 f   libsetfldw001.obj
 0001:0000079c       Java_nsk_jvmti_SetFieldAccessWatch_setfldw001_check 000000018000179c f   libsetfldw001.obj
 0001:00000818       Java_nsk_jvmti_SetFieldAccessWatch_setfldw001_getRes 0000000180001818 f   libsetfldw001.obj
 0001:00000820       Java_nsk_jvmti_SetFieldAccessWatch_setfldw001_setWatch 0000000180001820 f   libsetfldw001.obj
 0001:00000828       Java_nsk_jvmti_SetFieldAccessWatch_setfldw001_touchfld0 0000000180001828 f   libsetfldw001.obj
 0001:00000860       Java_nsk_jvmti_unit_FollowReferences_FollowRefObjects_addRefToVerify 0000000180001860 f   libsetfldw001.obj
 0001:00000a1c       Java_nsk_jvmti_unit_FollowReferences_FollowRefObjects_getTag 0000000180001a1c f   libsetfldw001.obj
 0001:00000ad8       Java_nsk_jvmti_unit_FollowReferences_FollowRefObjects_resetRefsToVerify 0000000180001ad8 f   libsetfldw001.obj
 0001:00000ae0       Java_nsk_jvmti_unit_FollowReferences_FollowRefObjects_resetTags 0000000180001ae0 f   libsetfldw001.obj
 0001:00000b24       Java_nsk_jvmti_unit_FollowReferences_FollowRefObjects_setTag 0000000180001b24 f   libsetfldw001.obj
 0001:00000d70       Java_nsk_share_jvmti_ArgumentHandler_getAgentOptionsString 0000000180001d70 f   libsetfldw001.obj
 0001:00000e1c       Java_nsk_share_jvmti_DebugeeClass_checkStatus 0000000180001e1c f   libsetfldw001.obj
 0001:00000ea4       Java_nsk_share_jvmti_DebugeeClass_resetAgentData 0000000180001ea4 f   libsetfldw001.obj
 0001:00000f04       Java_nsk_share_jvmti_RedefineAgent_agentStatus 0000000180001f04 f   libsetfldw001.obj
 0001:00000f10       Java_nsk_share_jvmti_RedefineAgent_isRedefined 0000000180001f10 f   libsetfldw001.obj
 0001:00000f1c       Java_nsk_share_jvmti_RedefineAgent_redefineAttempted 0000000180001f1c f   libsetfldw001.obj
 0001:00000f28       MA_checkStatus             0000000180001f28 f   libsetfldw001.obj
 0001:00000fcc       __local_stdio_printf_options 0000000180001fcc f i libsetfldw001.obj
 0001:0000119c       exitOnError                000000018000219c f   libsetfldw001.obj
 0001:00001250       fprintf                    0000000180002250 f i libsetfldw001.obj
 0001:00001294       nsk_jvmti_lverify          0000000180002294 f   libsetfldw001.obj
 0001:00001384       nsk_jvmti_resetAgentData   0000000180002384 f   libsetfldw001.obj
 0001:000013f8       nsk_lcomplain              00000001800023f8 f   libsetfldw001.obj
 0001:00001418       nsk_ldisplay               0000000180002418 f   libsetfldw001.obj
 0001:00001438       nsk_ltrace                 0000000180002438 f   libsetfldw001.obj
 0001:00001458       nsk_lvcomplain             0000000180002458 f   libsetfldw001.obj
 0001:00001610       nsk_lvdisplay              0000000180002610 f   libsetfldw001.obj
 0001:0000165c       nsk_lverify                000000018000265c f   libsetfldw001.obj
 0001:000016b8       nsk_lvtrace                00000001800026b8 f   libsetfldw001.obj
 0001:00001718       nsk_printf                 0000000180002718 f   libsetfldw001.obj
 0001:00001740       nsk_vprintf                0000000180002740 f   libsetfldw001.obj
 0001:000017f4       printf                     00000001800027f4 f i libsetfldw001.obj
 0001:00001848       setWatch                   0000000180002848 f   libsetfldw001.obj
 0001:00001e08       __raise_securityfailure    0000000180002e08 f   MSVCRT:gs_report.obj
 0001:00001e3c       __report_gsfailure         0000000180002e3c f   MSVCRT:gs_report.obj
 0001:0000207c       __GSHandlerCheck           000000018000307c f   MSVCRT:gshandler.obj
 0001:0000209c       __GSHandlerCheckCommon     000000018000309c f   MSVCRT:gshandler.obj
 0001:00002110       __security_check_cookie    0000000180003110 f   MSVCRT:amdsecgs.obj
 0001:00002450       _DllMainCRTStartup         0000000180003450 f   MSVCRT:dll_dllmain.obj
 0001:00002490       __scrt_acquire_startup_lock 0000000180003490 f   MSVCRT:utility.obj
 0001:000024cc       __scrt_dllmain_after_initialize_c 00000001800034cc f   MSVCRT:utility.obj
 0001:00002500       __scrt_dllmain_before_initialize_c 0000000180003500 f   MSVCRT:utility.obj
 0001:00002518       __scrt_dllmain_crt_thread_attach 0000000180003518 f   MSVCRT:utility.obj
 0001:00002540       __scrt_dllmain_crt_thread_detach 0000000180003540 f   MSVCRT:utility.obj
 0001:00002558       __scrt_dllmain_exception_filter 0000000180003558 f   MSVCRT:utility.obj
 0001:000025b8       __scrt_dllmain_uninitialize_c 00000001800035b8 f   MSVCRT:utility.obj
 0001:000025e8       __scrt_dllmain_uninitialize_critical 00000001800035e8 f   MSVCRT:utility.obj
 0001:000025fc       __scrt_initialize_crt      00000001800035fc f   MSVCRT:utility.obj
 0001:00002648       __scrt_initialize_onexit_tables 0000000180003648 f   MSVCRT:utility.obj
 0001:000026d4       __scrt_is_nonwritable_in_current_image 00000001800036d4 f   MSVCRT:utility.obj
 0001:0000276c       __scrt_release_startup_lock 000000018000376c f   MSVCRT:utility.obj
 0001:00002790       __scrt_uninitialize_crt    0000000180003790 f   MSVCRT:utility.obj
 0001:000027bc       _onexit                    00000001800037bc f   MSVCRT:utility.obj
 0001:000027f8       atexit                     00000001800037f8 f   MSVCRT:utility.obj
 0001:00002810       __crt_debugger_hook        0000000180003810 f   MSVCRT:utility_desktop.obj
 0001:00002818       __scrt_fastfail            0000000180003818 f   MSVCRT:utility_desktop.obj
 0001:00002964       _guard_check_icall_nop     0000000180003964 f i MSVCRT:guard_support.obj
 0001:00002968       __security_init_cookie     0000000180003968 f   MSVCRT:gs_support.obj
 0001:00002a14       DllMain                    0000000180003a14 f   MSVCRT:dll_dllmain_stub.obj
 0001:00002a38       ?__scrt_initialize_type_info@@YAXXZ 0000000180003a38 f   MSVCRT:tncleanup.obj
 0001:00002a48       ?__scrt_uninitialize_type_info@@YAXXZ 0000000180003a48 f   MSVCRT:tncleanup.obj
 0001:00002a54       __local_stdio_scanf_options 0000000180003a54 f i MSVCRT:default_local_stdio_options.obj
 0001:00002a5c       __scrt_initialize_default_local_stdio_options 0000000180003a5c f   MSVCRT:default_local_stdio_options.obj
 0001:00002a78       __scrt_get_dyn_tls_init_callback 0000000180003a78 f   MSVCRT:dyn_tls_init.obj
 0001:00002a80       _RTC_Initialize            0000000180003a80 f   MSVCRT:initsect.obj
 0001:00002abc       _RTC_Terminate             0000000180003abc f   MSVCRT:initsect.obj
 0001:00002af8       __isa_available_init       0000000180003af8 f   MSVCRT:cpu_disp.obj
 0001:00002ca4       _get_startup_argv_mode     0000000180003ca4 f   MSVCRT:argv_mode.obj
 0001:00002cac       __scrt_is_ucrt_dll_in_use  0000000180003cac f   MSVCRT:ucrt_detection.obj
 0001:00002cc0       memcpy                     0000000180003cc0 f   vcruntime:VCRUNTIME140.dll
 0001:00002cc6       memset                     0000000180003cc6 f   vcruntime:VCRUNTIME140.dll
 0001:00002ccc       strchr                     0000000180003ccc f   vcruntime:VCRUNTIME140.dll
 0001:00002cd2       __C_specific_handler       0000000180003cd2 f   vcruntime:VCRUNTIME140.dll
 0001:00002cd8       __std_type_info_destroy_list 0000000180003cd8 f   vcruntime:VCRUNTIME140.dll
 0001:00002cde       strlen                     0000000180003cde f   ucrt:api-ms-win-crt-string-l1-1-0.dll
 0001:00002ce4       _initterm                  0000000180003ce4 f   ucrt:api-ms-win-crt-runtime-l1-1-0.dll
 0001:00002cea       _initterm_e                0000000180003cea f   ucrt:api-ms-win-crt-runtime-l1-1-0.dll
 0001:00002cf0       _seh_filter_dll            0000000180003cf0 f   ucrt:api-ms-win-crt-runtime-l1-1-0.dll
 0001:00002cf6       _configure_narrow_argv     0000000180003cf6 f   ucrt:api-ms-win-crt-runtime-l1-1-0.dll
 0001:00002cfc       _initialize_narrow_environment 0000000180003cfc f   ucrt:api-ms-win-crt-runtime-l1-1-0.dll
 0001:00002d02       _initialize_onexit_table   0000000180003d02 f   ucrt:api-ms-win-crt-runtime-l1-1-0.dll
 0001:00002d08       _register_onexit_function  0000000180003d08 f   ucrt:api-ms-win-crt-runtime-l1-1-0.dll
 0001:00002d0e       _execute_onexit_table      0000000180003d0e f   ucrt:api-ms-win-crt-runtime-l1-1-0.dll
 0001:00002d14       _crt_atexit                0000000180003d14 f   ucrt:api-ms-win-crt-runtime-l1-1-0.dll
 0001:00002d1a       _cexit                     0000000180003d1a f   ucrt:api-ms-win-crt-runtime-l1-1-0.dll
 0001:00002d20       __acrt_initialize          0000000180003d20 f   MSVCRT:ucrt_stubs.obj
 0001:00002d20       __acrt_thread_attach       0000000180003d20 f   MSVCRT:ucrt_stubs.obj
 0001:00002d20       __acrt_thread_detach       0000000180003d20 f   MSVCRT:ucrt_stubs.obj
 0001:00002d20       __acrt_uninitialize        0000000180003d20 f   MSVCRT:ucrt_stubs.obj
 0001:00002d20       __acrt_uninitialize_critical 0000000180003d20 f   MSVCRT:ucrt_stubs.obj
 0001:00002d20       __scrt_stub_for_acrt_initialize 0000000180003d20 f   MSVCRT:ucrt_stubs.obj
 0001:00002d20       __scrt_stub_for_acrt_thread_attach 0000000180003d20 f   MSVCRT:ucrt_stubs.obj
 0001:00002d20       __scrt_stub_for_acrt_thread_detach 0000000180003d20 f   MSVCRT:ucrt_stubs.obj
 0001:00002d20       __scrt_stub_for_acrt_uninitialize 0000000180003d20 f   MSVCRT:ucrt_stubs.obj
 0001:00002d20       __scrt_stub_for_acrt_uninitialize_critical 0000000180003d20 f   MSVCRT:ucrt_stubs.obj
 0001:00002d20       __vcrt_initialize          0000000180003d20 f   MSVCRT:ucrt_stubs.obj
 0001:00002d20       __vcrt_thread_attach       0000000180003d20 f   MSVCRT:ucrt_stubs.obj
 0001:00002d20       __vcrt_thread_detach       0000000180003d20 f   MSVCRT:ucrt_stubs.obj
 0001:00002d20       __vcrt_uninitialize        0000000180003d20 f   MSVCRT:ucrt_stubs.obj
 0001:00002d20       __vcrt_uninitialize_critical 0000000180003d20 f   MSVCRT:ucrt_stubs.obj
 0001:00002d24       __scrt_stub_for_is_c_termination_complete 0000000180003d24 f   MSVCRT:ucrt_stubs.obj
 0001:00002d24       _is_c_termination_complete 0000000180003d24 f   MSVCRT:ucrt_stubs.obj
 0001:00002d40       _guard_dispatch_icall_nop  0000000180003d40 f   MSVCRT:guard_dispatch.obj
 0001:00002d60       _guard_xfg_dispatch_icall_nop 0000000180003d60 f   MSVCRT:guard_xfg_dispatch.obj
 0002:00000000       __imp_RtlCaptureContext    0000000180004000     kernel32:KERNEL32.dll
 0002:00000008       __imp_RtlLookupFunctionEntry 0000000180004008     kernel32:KERNEL32.dll
 0002:00000010       __imp_RtlVirtualUnwind     0000000180004010     kernel32:KERNEL32.dll
 0002:00000018       __imp_UnhandledExceptionFilter 0000000180004018     kernel32:KERNEL32.dll
 0002:00000020       __imp_SetUnhandledExceptionFilter 0000000180004020     kernel32:KERNEL32.dll
 0002:00000028       __imp_GetCurrentProcess    0000000180004028     kernel32:KERNEL32.dll
 0002:00000030       __imp_TerminateProcess     0000000180004030     kernel32:KERNEL32.dll
 0002:00000038       __imp_IsProcessorFeaturePresent 0000000180004038     kernel32:KERNEL32.dll
 0002:00000040       __imp_CloseHandle          0000000180004040     kernel32:KERNEL32.dll
 0002:00000048       __imp_InitializeCriticalSectionAndSpinCount 0000000180004048     kernel32:KERNEL32.dll
 0002:00000050       __imp_DeleteCriticalSection 0000000180004050     kernel32:KERNEL32.dll
 0002:00000058       __imp_CreateEventW         0000000180004058     kernel32:KERNEL32.dll
 0002:00000060       __imp_GetModuleHandleW     0000000180004060     kernel32:KERNEL32.dll
 0002:00000068       __imp_GetProcAddress       0000000180004068     kernel32:KERNEL32.dll
 0002:00000070       __imp_IsDebuggerPresent    0000000180004070     kernel32:KERNEL32.dll
 0002:00000078       __imp_QueryPerformanceCounter 0000000180004078     kernel32:KERNEL32.dll
 0002:00000080       __imp_GetCurrentProcessId  0000000180004080     kernel32:KERNEL32.dll
 0002:00000088       __imp_GetCurrentThreadId   0000000180004088     kernel32:KERNEL32.dll
 0002:00000090       __imp_GetSystemTimeAsFileTime 0000000180004090     kernel32:KERNEL32.dll
 0002:00000098       __imp_DisableThreadLibraryCalls 0000000180004098     kernel32:KERNEL32.dll
 0002:000000a0       __imp_InitializeSListHead  00000001800040a0     kernel32:KERNEL32.dll
 0002:000000a8       \177KERNEL32_NULL_THUNK_DATA 00000001800040a8     kernel32:KERNEL32.dll
 0002:000000b0       __imp_memcpy               00000001800040b0     vcruntime:VCRUNTIME140.dll
 0002:000000b8       __imp_memset               00000001800040b8     vcruntime:VCRUNTIME140.dll
 0002:000000c0       __imp_strchr               00000001800040c0     vcruntime:VCRUNTIME140.dll
 0002:000000c8       __imp___C_specific_handler 00000001800040c8     vcruntime:VCRUNTIME140.dll
 0002:000000d0       __imp___std_type_info_destroy_list 00000001800040d0     vcruntime:VCRUNTIME140.dll
 0002:000000d8       \177VCRUNTIME140_NULL_THUNK_DATA 00000001800040d8     vcruntime:VCRUNTIME140.dll
 0002:000000e0       __imp__errno               00000001800040e0     ucrt:api-ms-win-crt-runtime-l1-1-0.dll
 0002:000000e8       __imp_exit                 00000001800040e8     ucrt:api-ms-win-crt-runtime-l1-1-0.dll
 0002:000000f0       __imp__cexit               00000001800040f0     ucrt:api-ms-win-crt-runtime-l1-1-0.dll
 0002:000000f8       __imp__crt_atexit          00000001800040f8     ucrt:api-ms-win-crt-runtime-l1-1-0.dll
 0002:00000100       __imp__execute_onexit_table 0000000180004100     ucrt:api-ms-win-crt-runtime-l1-1-0.dll
 0002:00000108       __imp__register_onexit_function 0000000180004108     ucrt:api-ms-win-crt-runtime-l1-1-0.dll
 0002:00000110       __imp__initialize_onexit_table 0000000180004110     ucrt:api-ms-win-crt-runtime-l1-1-0.dll
 0002:00000118       __imp__initialize_narrow_environment 0000000180004118     ucrt:api-ms-win-crt-runtime-l1-1-0.dll
 0002:00000120       __imp__configure_narrow_argv 0000000180004120     ucrt:api-ms-win-crt-runtime-l1-1-0.dll
 0002:00000128       __imp__seh_filter_dll      0000000180004128     ucrt:api-ms-win-crt-runtime-l1-1-0.dll
 0002:00000130       __imp__initterm_e          0000000180004130     ucrt:api-ms-win-crt-runtime-l1-1-0.dll
 0002:00000138       __imp__initterm            0000000180004138     ucrt:api-ms-win-crt-runtime-l1-1-0.dll
 0002:00000140       \177api-ms-win-crt-runtime-l1-1-0_NULL_THUNK_DATA 0000000180004140     ucrt:api-ms-win-crt-runtime-l1-1-0.dll
 0002:00000148       __imp___acrt_iob_func      0000000180004148     ucrt:api-ms-win-crt-stdio-l1-1-0.dll
 0002:00000150       __imp_fflush               0000000180004150     ucrt:api-ms-win-crt-stdio-l1-1-0.dll
 0002:00000158       __imp___stdio_common_vsprintf 0000000180004158     ucrt:api-ms-win-crt-stdio-l1-1-0.dll
 0002:00000160       __imp___stdio_common_vfprintf 0000000180004160     ucrt:api-ms-win-crt-stdio-l1-1-0.dll
 0002:00000168       \177api-ms-win-crt-stdio-l1-1-0_NULL_THUNK_DATA 0000000180004168     ucrt:api-ms-win-crt-stdio-l1-1-0.dll
 0002:00000170       __imp_isdigit              0000000180004170     ucrt:api-ms-win-crt-string-l1-1-0.dll
 0002:00000178       __imp__strdup              0000000180004178     ucrt:api-ms-win-crt-string-l1-1-0.dll
 0002:00000178       __imp_strdup               0000000180004178     ucrt:api-ms-win-crt-string-l1-1-0.dll
 0002:00000180       __imp_strlen               0000000180004180     ucrt:api-ms-win-crt-string-l1-1-0.dll
 0002:00000188       __imp_strncpy              0000000180004188     ucrt:api-ms-win-crt-string-l1-1-0.dll
 0002:00000190       \177api-ms-win-crt-string-l1-1-0_NULL_THUNK_DATA 0000000180004190     ucrt:api-ms-win-crt-string-l1-1-0.dll
 0002:00000198       __guard_check_icall_fptr   0000000180004198     MSVCRT:guard_support.obj
 0002:000001a0       __guard_xfg_check_icall_fptr 00000001800041a0     MSVCRT:guard_support.obj
 0002:000001a8       __guard_dispatch_icall_fptr 00000001800041a8     MSVCRT:guard_support.obj
 0002:000001b0       __guard_xfg_dispatch_icall_fptr 00000001800041b0     MSVCRT:guard_support.obj
 0002:000001b8       __guard_xfg_table_dispatch_icall_fptr 00000001800041b8     MSVCRT:guard_support.obj
 0002:000001c0       __castguard_check_failure_os_handled_fptr 00000001800041c0     MSVCRT:guard_support.obj
 0002:000001c8       __guard_memcpy_fptr        00000001800041c8     vcruntime:softmemtag.obj
 0002:000001d0       __xc_a                     00000001800041d0     MSVCRT:initializers.obj
 0002:000001d8       __xc_z                     00000001800041d8     MSVCRT:initializers.obj
 0002:000001e0       __xi_a                     00000001800041e0     MSVCRT:initializers.obj
 0002:000001f0       __xi_z                     00000001800041f0     MSVCRT:initializers.obj
 0002:000001f8       __xl_a                     00000001800041f8     MSVCRT:tlssup.obj
 0002:00000200       __xl_z                     0000000180004200     MSVCRT:tlssup.obj
 0002:00000208       __xp_a                     0000000180004208     MSVCRT:initializers.obj
 0002:00000210       __xp_z                     0000000180004210     MSVCRT:initializers.obj
 0002:00000218       __xt_a                     0000000180004218     MSVCRT:initializers.obj
 0002:00000220       __xt_z                     0000000180004220     MSVCRT:initializers.obj
 0002:00000230       g_refKindStr               0000000180004230     libsetfldw001.obj
 0002:000003e0       ??_C@_09BPLDFGCI@unknown_0@ 00000001800043e0     libsetfldw001.obj
 0002:000003f0       ??_C@_0BL@FPNMECJD@JVMTI_HEAP_REFERENCE_CLASS@ 00000001800043f0     libsetfldw001.obj
 0002:00000410       ??_C@_0BL@FKGKKLNM@JVMTI_HEAP_REFERENCE_FIELD@ 0000000180004410     libsetfldw001.obj
 0002:00000430       ??_C@_0CD@CAEHCFJF@JVMTI_HEAP_REFERENCE_ARRAY_ELEM@ 0000000180004430     libsetfldw001.obj
 0002:00000458       ??_C@_0CC@DNEBMCNK@JVMTI_HEAP_REFERENCE_CLASS_LOAD@ 0000000180004458     libsetfldw001.obj
 0002:00000480       ??_C@_0BN@CJMIPEBB@JVMTI_HEAP_REFERENCE_SIGNERS@ 0000000180004480     libsetfldw001.obj
 0002:000004a0       ??_C@_0CH@HBOIDPEB@JVMTI_HEAP_REFERENCE_PROTECTION@ 00000001800044a0     libsetfldw001.obj
 0002:000004c8       ??_C@_0BP@MDKGDGKL@JVMTI_HEAP_REFERENCE_INTERFACE@ 00000001800044c8     libsetfldw001.obj
 0002:000004e8       ??_C@_0CC@JJMIHNJH@JVMTI_HEAP_REFERENCE_STATIC_FIE@ 00000001800044e8     libsetfldw001.obj
 0002:00000510       ??_C@_0CD@IDHEEGID@JVMTI_HEAP_REFERENCE_CONSTANT_P@ 0000000180004510     libsetfldw001.obj
 0002:00000538       ??_C@_0CA@EFFCHNG@JVMTI_HEAP_REFERENCE_SUPERCLASS@ 0000000180004538     libsetfldw001.obj
 0002:00000558       ??_C@_0L@PCDFHGCJ@unknown_11@ 0000000180004558     libsetfldw001.obj
 0002:00000568       ??_C@_0L@NJBICFOK@unknown_12@ 0000000180004568     libsetfldw001.obj
 0002:00000578       ??_C@_0L@MAADBEKL@unknown_13@ 0000000180004578     libsetfldw001.obj
 0002:00000588       ??_C@_0L@IPECICGM@unknown_14@ 0000000180004588     libsetfldw001.obj
 0002:00000598       ??_C@_0L@JGFJLDCN@unknown_15@ 0000000180004598     libsetfldw001.obj
 0002:000005a8       ??_C@_0L@LNHEOAOO@unknown_16@ 00000001800045a8     libsetfldw001.obj
 0002:000005b8       ??_C@_0L@KEGPNBKP@unknown_17@ 00000001800045b8     libsetfldw001.obj
 0002:000005c8       ??_C@_0L@CDPHMNGA@unknown_18@ 00000001800045c8     libsetfldw001.obj
 0002:000005d8       ??_C@_0L@DKOMPMCB@unknown_19@ 00000001800045d8     libsetfldw001.obj
 0002:000005e8       ??_C@_0L@OJGIPJDB@unknown_20@ 00000001800045e8     libsetfldw001.obj
 0002:000005f8       ??_C@_0CA@KAOFNDEM@JVMTI_HEAP_REFERENCE_JNI_GLOBAL@ 00000001800045f8     libsetfldw001.obj
 0002:00000618       ??_C@_0CC@HPFAJBK@JVMTI_HEAP_REFERENCE_SYSTEM_CLA@ 0000000180004618     libsetfldw001.obj
 0002:00000640       ??_C@_0BN@FDEGFOHC@JVMTI_HEAP_REFERENCE_MONITOR@ 0000000180004640     libsetfldw001.obj
 0002:00000660       ??_C@_0CB@HKIBCMAJ@JVMTI_HEAP_REFERENCE_STACK_LOCA@ 0000000180004660     libsetfldw001.obj
 0002:00000688       ??_C@_0BP@EAACMMOE@JVMTI_HEAP_REFERENCE_JNI_LOCAL@ 0000000180004688     libsetfldw001.obj
 0002:000006a8       ??_C@_0BM@IJDEOGOE@JVMTI_HEAP_REFERENCE_THREAD@ 00000001800046a8     libsetfldw001.obj
 0002:000006c8       ??_C@_0BL@EDGPPKC@JVMTI_HEAP_REFERENCE_OTHER@ 00000001800046c8     libsetfldw001.obj
 0002:000006e4       ??_C@_04BCJPDBDA@Code@     00000001800046e4     libsetfldw001.obj
 0002:000006f0       ??_C@_0BA@OCLMCFKC@LineNumberTable@ 00000001800046f0     libsetfldw001.obj
 0002:00000700       ??_C@_0BD@CPAEPILC@LocalVariableTable@ 0000000180004700     libsetfldw001.obj
 0002:00000718       ??_C@_0BH@NMBDNHBD@LocalVariableTypeTable@ 0000000180004718     libsetfldw001.obj
 0002:00000730       ??_C@_0O@HIHEEDNJ@StackMapTable@ 0000000180004730     libsetfldw001.obj
 0002:00000740       ??_C@_0CJ@IHJGEIDH@nsk?1jvmti?1SetFieldAccessWatch?1s@ 0000000180004740     libsetfldw001.obj
 0002:0000076c       ??_C@_04MOMHJHLL@fld0@     000000018000476c     libsetfldw001.obj
 0002:00000774       ??_C@_01JPJNBJEM@I@        0000000180004774     libsetfldw001.obj
 0002:00000778       ??_C@_04NHNMKGPK@fld1@     0000000180004778     libsetfldw001.obj
 0002:00000780       ??_C@_04PMPBPFDJ@fld2@     0000000180004780     libsetfldw001.obj
 0002:00000788       ??_C@_0CM@EODKHGNF@Lnsk?1jvmti?1SetFieldAccessWatch?1@ 0000000180004788     libsetfldw001.obj
 0002:000007b8       ??_C@_0CK@MENMGJKB@nsk?1jvmti?1SetFieldAccessWatch?1s@ 00000001800047b8     libsetfldw001.obj
 0002:000007e4       ??_C@_04OFOKMEHI@fld3@     00000001800047e4     libsetfldw001.obj
 0002:000007ec       ??_C@_02EBOMBDPA@?$FLI@    00000001800047ec     libsetfldw001.obj
 0002:000007f0       ??_C@_0CK@OPPBDKGC@nsk?1jvmti?1SetFieldAccessWatch?1s@ 00000001800047f0     libsetfldw001.obj
 0002:0000081c       ??_C@_04KKKLFCLP@fld4@     000000018000481c     libsetfldw001.obj
 0002:00000824       ??_C@_01BIAFAFID@F@        0000000180004824     libsetfldw001.obj
 0002:00000828       ??_C@_0L@HCDIAMJG@?9?5?$CFs?0?5?$CFd?3?5@ 0000000180004828     libsetfldw001.obj
 0002:00000840       ??_C@_0JI@HLPECLFI@?$CD?5?4?4?4?6?$CD?5ERROR?3?5too?5many?5complai@ 0000000180004840     libsetfldw001.obj
 0002:000008e0       ??_C@_0ED@JNEKCCOB@The?5following?5fake?5exception?5st@ 00000001800048e0     libsetfldw001.obj
 0002:00000928       ??_C@_0CN@FCNMDFBH@nsk?4share?4Fake_Exception_for_RU@ 0000000180004928     libsetfldw001.obj
 0002:00000958       ??_C@_08PGFFNAEI@?$CI?$CFs?3?$CFd?$CJ?5@ 0000000180004958     libsetfldw001.obj
 0002:00000968       ??_C@_0DP@IENMAEGI@s?2test?2hotspot?2jtreg?2vmTestbase@ 0000000180004968     libsetfldw001.obj
 0002:000009a8       ??_C@_0BL@NDJLFFJB@?7at?5nsk_lvcomplain?$CI?$CFs?3?$CFd?$CJ?6@ 00000001800049a8     libsetfldw001.obj
 0002:000009c8       ??_C@_0BC@JOOKAFKF@?$CD?5ERROR?3?5?$CFs?0?5?$CFd?3?5@ 00000001800049c8     libsetfldw001.obj
 0002:000009e0       ??_C@_09KJEAHMEH@?$CD?5ERROR?3?5@ 00000001800049e0     libsetfldw001.obj
 0002:000009ec       ??_C@_02GPIOPFAK@?$DO?$DO@ 00000001800049ec     libsetfldw001.obj
 0002:000009f0       ??_C@_02FODMEDOG@?$DM?$DM@ 00000001800049f0     libsetfldw001.obj
 0002:000009f4       ??_C@_02DJGKEECL@?4?4@     00000001800049f4     libsetfldw001.obj
 0002:000009f8       ??_C@_0O@CJPGJOAF@?9?5?$CFs?0?5?$CFd?3?5?$CFs?5@ 00000001800049f8     libsetfldw001.obj
 0002:00000a08       ??_C@_0CB@IAKPDOIC@?$CD?5?5?5verified?5assertion?5is?5FALSE@ 0000000180004a08     libsetfldw001.obj
 0002:00000a30       ??_C@_0CO@LGONDEPD@stdout?3?5fflush?5failed?5?9?5err?$DN?$CFd?5@ 0000000180004a30     libsetfldw001.obj
 0002:00000a60       ??_C@_0CO@KBGKJPBD@stderr?3?5fflush?5failed?5?9?5err?$DN?$CFd?5@ 0000000180004a60     libsetfldw001.obj
 0002:00000a90       ??_C@_0BB@JCNMKLLK@JVMTI_ERROR_NONE@ 0000000180004a90     libsetfldw001.obj
 0002:00000aa8       ??_C@_0BL@LDIMKLPH@JVMTI_ERROR_INVALID_THREAD@ 0000000180004aa8     libsetfldw001.obj
 0002:00000ac8       ??_C@_0CB@PJFPAIKJ@JVMTI_ERROR_INVALID_THREAD_GROU@ 0000000180004ac8     libsetfldw001.obj
 0002:00000af0       ??_C@_0BN@LLMKHMNF@JVMTI_ERROR_INVALID_PRIORITY@ 0000000180004af0     libsetfldw001.obj
 0002:00000b10       ??_C@_0CB@MBOFKAGB@JVMTI_ERROR_THREAD_NOT_SUSPENDE@ 0000000180004b10     libsetfldw001.obj
 0002:00000b38       ??_C@_0BN@FABOLPBI@JVMTI_ERROR_THREAD_SUSPENDED@ 0000000180004b38     libsetfldw001.obj
 0002:00000b58       ??_C@_0BN@FDGNOBJM@JVMTI_ERROR_THREAD_NOT_ALIVE@ 0000000180004b58     libsetfldw001.obj
 0002:00000b78       ??_C@_0BL@GOBIFKNJ@JVMTI_ERROR_INVALID_OBJECT@ 0000000180004b78     libsetfldw001.obj
 0002:00000b98       ??_C@_0BK@FCMAJPPC@JVMTI_ERROR_INVALID_CLASS@ 0000000180004b98     libsetfldw001.obj
 0002:00000bb8       ??_C@_0BP@IKLLBKEB@JVMTI_ERROR_CLASS_NOT_PREPARED@ 0000000180004bb8     libsetfldw001.obj
 0002:00000bd8       ??_C@_0BN@KLPPLKG@JVMTI_ERROR_INVALID_METHODID@ 0000000180004bd8     libsetfldw001.obj
 0002:00000bf8       ??_C@_0BN@BCEKOKND@JVMTI_ERROR_INVALID_LOCATION@ 0000000180004bf8     libsetfldw001.obj
 0002:00000c18       ??_C@_0BM@DFDGPME@JVMTI_ERROR_INVALID_FIELDID@ 0000000180004c18     libsetfldw001.obj
 0002:00000c38       ??_C@_0BL@NELIEPEC@JVMTI_ERROR_NO_MORE_FRAMES@ 0000000180004c38     libsetfldw001.obj
 0002:00000c58       ??_C@_0BJ@BDBECFDM@JVMTI_ERROR_OPAQUE_FRAME@ 0000000180004c58     libsetfldw001.obj
 0002:00000c78       ??_C@_0BK@MIIFNLOB@JVMTI_ERROR_TYPE_MISMATCH@ 0000000180004c78     libsetfldw001.obj
 0002:00000c98       ??_C@_0BJ@HPCAOILC@JVMTI_ERROR_INVALID_SLOT@ 0000000180004c98     libsetfldw001.obj
 0002:00000cb8       ??_C@_0BG@CHILOPNI@JVMTI_ERROR_DUPLICATE@ 0000000180004cb8     libsetfldw001.obj
 0002:00000cd0       ??_C@_0BG@DIEMLHKM@JVMTI_ERROR_NOT_FOUND@ 0000000180004cd0     libsetfldw001.obj
 0002:00000ce8       ??_C@_0BM@NHMCKHOB@JVMTI_ERROR_INVALID_MONITOR@ 0000000180004ce8     libsetfldw001.obj
 0002:00000d08       ??_C@_0BO@PPEDAJGL@JVMTI_ERROR_NOT_MONITOR_OWNER@ 0000000180004d08     libsetfldw001.obj
 0002:00000d28       ??_C@_0BG@FCAIPEID@JVMTI_ERROR_INTERRUPT@ 0000000180004d28     libsetfldw001.obj
 0002:00000d40       ??_C@_0CB@EGDBNKOI@JVMTI_ERROR_INVALID_CLASS_FORMA@ 0000000180004d40     libsetfldw001.obj
 0002:00000d68       ??_C@_0CG@DGKOGIAL@JVMTI_ERROR_CIRCULAR_CLASS_DEFI@ 0000000180004d68     libsetfldw001.obj
 0002:00000d90       ??_C@_0BP@ICEALPKC@JVMTI_ERROR_FAILS_VERIFICATION@ 0000000180004d90     libsetfldw001.obj
 0002:00000db0       ??_C@_0DC@JDACLMIO@JVMTI_ERROR_UNSUPPORTED_REDEFIN@ 0000000180004db0     libsetfldw001.obj
 0002:00000de8       ??_C@_0DE@GKDKNOMJ@JVMTI_ERROR_UNSUPPORTED_REDEFIN@ 0000000180004de8     libsetfldw001.obj
 0002:00000e20       ??_C@_0BO@LAFKIOG@JVMTI_ERROR_INVALID_TYPESTATE@ 0000000180004e20     libsetfldw001.obj
 0002:00000e40       ??_C@_0DH@INDGCLLB@JVMTI_ERROR_UNSUPPORTED_REDEFIN@ 0000000180004e40     libsetfldw001.obj
 0002:00000e78       ??_C@_0DE@NHEOMMGI@JVMTI_ERROR_UNSUPPORTED_REDEFIN@ 0000000180004e78     libsetfldw001.obj
 0002:00000eb0       ??_C@_0CA@EKPNJOEP@JVMTI_ERROR_UNSUPPORTED_VERSION@ 0000000180004eb0     libsetfldw001.obj
 0002:00000ed0       ??_C@_0BN@OFFMAHHL@JVMTI_ERROR_NAMES_DONT_MATCH@ 0000000180004ed0     libsetfldw001.obj
 0002:00000ef0       ??_C@_0DN@HHBBLAKE@JVMTI_ERROR_UNSUPPORTED_REDEFIN@ 0000000180004ef0     libsetfldw001.obj
 0002:00000f30       ??_C@_0DO@HMBGBGNA@JVMTI_ERROR_UNSUPPORTED_REDEFIN@ 0000000180004f30     libsetfldw001.obj
 0002:00000f70       ??_C@_0BP@PBECGKHJ@JVMTI_ERROR_UNMODIFIABLE_CLASS@ 0000000180004f70     libsetfldw001.obj
 0002:00000f90       ??_C@_0BK@CANILEHF@JVMTI_ERROR_NOT_AVAILABLE@ 0000000180004f90     libsetfldw001.obj
 0002:00000fb0       ??_C@_0CE@INJKMEFK@JVMTI_ERROR_MUST_POSSESS_CAPABI@ 0000000180004fb0     libsetfldw001.obj
 0002:00000fd8       ??_C@_0BJ@LBFPFPDM@JVMTI_ERROR_NULL_POINTER@ 0000000180004fd8     libsetfldw001.obj
 0002:00000ff8       ??_C@_0BP@CHJPNNEM@JVMTI_ERROR_ABSENT_INFORMATION@ 0000000180004ff8     libsetfldw001.obj
 0002:00001018       ??_C@_0BP@OMFMNLC@JVMTI_ERROR_INVALID_EVENT_TYPE@ 0000000180005018     libsetfldw001.obj
 0002:00001038       ??_C@_0BN@BIBNPHHO@JVMTI_ERROR_ILLEGAL_ARGUMENT@ 0000000180005038     libsetfldw001.obj
 0002:00001058       ??_C@_0BK@KKNDHDCE@JVMTI_ERROR_NATIVE_METHOD@ 0000000180005058     libsetfldw001.obj
 0002:00001078       ??_C@_0BK@PMKCFHAE@JVMTI_ERROR_OUT_OF_MEMORY@ 0000000180005078     libsetfldw001.obj
 0002:00001098       ??_C@_0BK@NNJBDMNB@JVMTI_ERROR_ACCESS_DENIED@ 0000000180005098     libsetfldw001.obj
 0002:000010b8       ??_C@_0BI@GHECLMNC@JVMTI_ERROR_WRONG_PHASE@ 00000001800050b8     libsetfldw001.obj
 0002:000010d0       ??_C@_0BF@OLIHJOII@JVMTI_ERROR_INTERNAL@ 00000001800050d0     libsetfldw001.obj
 0002:000010e8       ??_C@_0BO@EOHGKJHI@JVMTI_ERROR_UNATTACHED_THREAD@ 00000001800050e8     libsetfldw001.obj
 0002:00001108       ??_C@_0CA@LKHFDACL@JVMTI_ERROR_INVALID_ENVIRONMENT@ 0000000180005108     libsetfldw001.obj
 0002:00001128       ??_C@_0BA@MMFHLOKK@?$DMunknown?5error?$DO@ 0000000180005128     libsetfldw001.obj
 0002:00001138       ??_C@_0CF@CBHOKDB@throwable?5?$DN?5jni?9?$DOExceptionOccur@ 0000000180005138     libsetfldw001.obj
 0002:00001160       ??_C@_03OFAPEBGM@?$CFs?6@  0000000180005160     libsetfldw001.obj
 0002:00001168       ??_C@_0DM@LPIGEGNJ@s?2test?2hotspot?2jtreg?2vmTestbase@ 0000000180005168     libsetfldw001.obj
 0002:000011a8       ??_C@_0CC@NFCNPEPK@Exception?5in?5JNI?5call?5?$CIcleared?$CJ@ 00000001800051a8     libsetfldw001.obj
 0002:000011d0       ??_C@_0BJ@IBAKFIKF@jni?9?$DOExceptionDescribe?$CI?$CJ@ 00000001800051d0     libsetfldw001.obj
 0002:000011f0       ??_C@_0BG@GGKALKMH@jni?9?$DOExceptionClear?$CI?$CJ@ 00000001800051f0     libsetfldw001.obj
 0002:00001208       ??_C@_0CF@JMGFGJLJ@?$CD?5?5?5verified?5JNI?5assertion?5is?5F@ 0000000180005208     libsetfldw001.obj
 0002:00001230       ??_C@_0CB@MLNJNCLJ@?5?5jvmti?5error?3?5code?$DN?$CFd?0?5name?$DN?$CFs@ 0000000180005230     libsetfldw001.obj
 0002:00001258       ??_C@_0CD@OHBGDKMK@?$CD?5?5?5jvmti?5error?3?5code?$DN?$CFd?0?5name?$DN@ 0000000180005258     libsetfldw001.obj
 0002:00001280       ??_C@_0CG@JNNCGPHB@?$CD?5?5?5error?5expected?3?5code?$DN?$CFd?0?5na@ 0000000180005280     libsetfldw001.obj
 0002:000012b0       ??_C@_0EB@IMGKPCGE@?$CIstr_obj?5?$DN?5jni?9?$DONewStringUTF?$CIco@ 00000001800052b0     libsetfldw001.obj
 0002:00001300       ??_C@_0EA@HFOGGBCC@s?2test?2hotspot?2jtreg?2vmTestbase@ 0000000180005300     libsetfldw001.obj
 0002:00001340       ??_C@_05KKCIMGE@error@     0000000180005340     libsetfldw001.obj
 0002:00001350       ??_C@_0EA@PNBCDMOA@s?2test?2hotspot?2jtreg?2vmTestbase@ 0000000180005350     libsetfldw001.obj
 0002:00001390       ??_C@_0DI@ILAHDLMP@?$CI?$CKagentThreadProc?$CJ?$CIjvmti_env?0?5a@ 0000000180005390     libsetfldw001.obj
 0002:000013c8       ??_C@_0BD@KDBALNLB@JVMTI?5agent?5thread@ 00000001800053c8     libsetfldw001.obj
 0002:000013e0       ??_C@_0BB@NOKBFPFO@java?1lang?1Thread@ 00000001800053e0     libsetfldw001.obj
 0002:000013f4       ??_C@_06FALKBLGB@?$DMinit?$DO@ 00000001800053f4     libsetfldw001.obj
 0002:00001400       ??_C@_0BG@IKDDPPGD@?$CILjava?1lang?1String?$DL?$CJV@ 0000000180005400     libsetfldw001.obj
 0002:00001420       ??_C@_0EB@IFJBFEKC@?$CIthreadClass?5?$DN?5jni_env?9?$DOFindCla@ 0000000180005420     libsetfldw001.obj
 0002:00001470       ??_C@_0GF@FGFIBKKL@?$CIthreadCtor?5?$DN?5jni_env?9?$DOGetMetho@ 0000000180005470     libsetfldw001.obj
 0002:000014d8       ??_C@_0DN@NCPDJLOG@?$CIthreadName?5?$DN?5jni_env?9?$DONewStrin@ 00000001800054d8     libsetfldw001.obj
 0002:00001520       ??_C@_0FE@PFKODBGC@?$CIthreadObject?5?$DN?5jni_env?9?$DONewObj@ 0000000180005520     libsetfldw001.obj
 0002:00001580       ??_C@_0ED@HOBAHHJI@?$CIthreadGlobalRef?5?$DN?5jni_env?9?$DONew@ 0000000180005580     libsetfldw001.obj
 0002:000015d0       ??_C@_0FN@HNJJAHFC@jvmti_env?9?$DORunAgentThread?$CIagent@ 00000001800055d0     libsetfldw001.obj
 0002:00001630       ??_C@_0EA@MOJDNKDF@Debuggee?5status?5sync?5aborted?5be@ 0000000180005630     libsetfldw001.obj
 0002:00001670       ??_C@_0EA@EEOEJAEN@status?5?$DN?5syncDebuggeeStatus?$CIjni@ 0000000180005670     libsetfldw001.obj
 0002:000016b0       ??_C@_0BL@JBCFNBMB@nsk_jvmti_resetAgentData?$CI?$CJ@ 00000001800056b0     libsetfldw001.obj
 0002:000016d0       ??_C@_0EL@LPBEELIP@s?2test?2hotspot?2jtreg?2vmTestbase@ 00000001800056d0     libsetfldw001.obj
 0002:00001720       ??_C@_0CK@JDAMFDMJ@jvmti?9?$DOSetTag?$CIo?0?5tag?$CJ?5?$DN?$DN?5JVMTI_@ 0000000180005720     libsetfldw001.obj
 0002:00001750       ??_C@_0CC@DAMNHKNI@Can?8t?5set?5tag?5?$CFli?5for?5object?5?$CFl@ 0000000180005750     libsetfldw001.obj
 0002:00001778       ??_C@_0DL@HAJPNKEF@jvmti?9?$DOGetObjectHashCode?$CIo?0?5?$CGha@ 0000000180005778     libsetfldw001.obj
 0002:000017b8       ??_C@_0BL@JFPIEOBF@Can?8t?5get?5hash?5object?5?$CFlx?6@ 00000001800057b8     libsetfldw001.obj
 0002:000017d8       ??_C@_0BG@DICPHBKN@setTag?3?5?$CF08x?5?$DM?9?5?$CF?53li@ 00000001800057d8     libsetfldw001.obj
 0002:000017f0       ??_C@_0DH@FCEEBDMJ@?$CIs?5?$DN?5jni?9?$DOGetStringUTFChars?$CIsIn@ 00000001800057f0     libsetfldw001.obj
 0002:00001828       ??_C@_0BJ@OKKGHDCN@Can?8t?5get?5string?5at?5?$CF?$CDp?6@ 0000000180005828     libsetfldw001.obj
 0002:00001848       ??_C@_0BP@EKFLGGFJ@Can?8t?5get?5string?5at?5?$CF?$CDp?3?5null?6@ 0000000180005848     libsetfldw001.obj
 0002:00001868       ??_C@_06ICODBHCL@?5?1?1?5?$CFs@ 0000000180005868     libsetfldw001.obj
 0002:00001870       ??_C@_0DB@KGFPLEGO@?$CIr?5?$DN?5jvmti?9?$DOGetTag?$CIo?0?5?$CGtag?$CJ?$CJ?5?$DN?$DN@ 0000000180005870     libsetfldw001.obj
 0002:000018a8       ??_C@_0CO@PDAGBCGJ@Can?8t?5GetTag?5for?5object?5?$CFlx?4?5Re@ 00000001800058a8     libsetfldw001.obj
 0002:000018d8       ??_C@_0CH@HPEODOHC@TEST_BUG?3?5Max?4?5number?5of?5refs?5r@ 00000001800058d8     libsetfldw001.obj
 0002:00001900       ??_C@_0DI@PHFCABIM@?$CIr?5?$DN?5jvmti?9?$DOGetTag?$CIfrom?0?5?$CGtagFr@ 0000000180005900     libsetfldw001.obj
 0002:00001938       ??_C@_0DI@MDEGFNKD@TEST_BUG?3?5Can?8t?5GetTag?5for?5obje@ 0000000180005938     libsetfldw001.obj
 0002:00001970       ??_C@_0DE@MLELJAHM@?$CIr?5?$DN?5jvmti?9?$DOGetTag?$CIto?0?5?$CGtagTo?$CJ?$CJ@ 0000000180005970     libsetfldw001.obj
 0002:000019a8       ??_C@_0BI@EFHFCFHM@Cannot?5find?5class?5?$CC?$CFs?$CC?6@ 00000001800059a8     libsetfldw001.obj
 0002:000019c0       ??_C@_0DE@NLBAFBC@?$CISetFieldAccessWatch?$CD?$CFd?$CJ?5unexpe@ 00000001800059c0     libsetfldw001.obj
 0002:000019f8       ??_C@_0CA@OJKPCPLI@Error?5in?5GetFieldName?3?5?$CFs?5?$CI?$CFd?$CJ?6@ 00000001800059f8     libsetfldw001.obj
 0002:00001a18       ??_C@_0CH@JDCHCCOE@GetFieldName?5returned?5null?5fiel@ 0000000180005a18     libsetfldw001.obj
 0002:00001a40       ??_C@_0DB@KDEBHECJ@GetFieldName?5returned?5unexpecte@ 0000000180005a40     libsetfldw001.obj
 0002:00001a78       ??_C@_0CK@NCAIGNEI@null?5field?5ID?5in?5FieldModificat@ 0000000180005a78     libsetfldw001.obj
 0002:00001aa8       ??_C@_0DG@GHLCFEDL@Event?3?5?$CIField?5?$CFd?$CJ?5field?5ID?5expe@ 0000000180005aa8     libsetfldw001.obj
 0002:00001ae0       ??_C@_0CK@DEFLIKCM@Wrong?5result?5of?5a?5valid?5call?5to@ 0000000180005ae0     libsetfldw001.obj
 0002:00001b10       ??_C@_0DG@LAJPGIIE@?$CIGetPotentialCapabilities?$CJ?5unex@ 0000000180005b10     libsetfldw001.obj
 0002:00001b48       ??_C@_0CN@LKPEOJPO@?$CIAddCapabilities?$CJ?5unexpected?5er@ 0000000180005b48     libsetfldw001.obj
 0002:00001b78       ??_C@_0CN@BCCBOHCH@?$CIGetCapabilities?$CJ?5unexpected?5er@ 0000000180005b78     libsetfldw001.obj
 0002:00001ba8       ??_C@_0CP@IMINGNLL@?$CISetEventCallbacks?$CJ?5unexpected?5@ 0000000180005ba8     libsetfldw001.obj
 0002:00001bd8       ??_C@_0DE@KEHGMPPJ@Failed?5to?5enable?5JVMTI_EVENT_FI@ 0000000180005bd8     libsetfldw001.obj
 0002:00001c10       ??_C@_0CP@EICFDPOA@Warning?3?5FieldAccess?5watch?5is?5n@ 0000000180005c10     libsetfldw001.obj
 0002:00001c40       ??_C@_0DI@JECEAFJC@?$CIField?5?$CFd?$CJ?5FIELD_ACCESS?5event?5w@ 0000000180005c40     libsetfldw001.obj
 0002:00001c78       ??_C@_0DG@NAFMPMGP@?$CIField?5?$CFd?$CJ?5thrown?5field?5ID?5expe@ 0000000180005c78     libsetfldw001.obj
 0002:00001cc0       ??_C@_1EC@JIJBPKFM@?$AAa?$AAp?$AAi?$AA?9?$AAm?$AAs?$AA?9?$AAw?$AAi?$AAn?$AA?9?$AAc?$AAo?$AAr?$AAe@ 0000000180005cc0     MSVCRT:thread_safe_statics.obj
 0002:00001d08       ??_C@_1BK@MGMFAEKH@?$AAk?$AAe?$AAr?$AAn?$AAe?$AAl?$AA3?$AA2?$AA?4?$AAd?$AAl?$AAl@ 0000000180005d08     MSVCRT:thread_safe_statics.obj
 0002:00001d28       ??_C@_0BJ@JEBJOJFJ@SleepConditionVariableCS@ 0000000180005d28     MSVCRT:thread_safe_statics.obj
 0002:00001d48       ??_C@_0BJ@PGPPEPCC@WakeAllConditionVariable@ 0000000180005d48     MSVCRT:thread_safe_statics.obj
 0002:00001d68       _pDefaultRawDllMain        0000000180005d68     MSVCRT:dll_dllmain.obj
 0002:00001d68       _pRawDllMain               0000000180005d68     MSVCRT:dll_dllmain.obj
 0002:00001d70       __xmm@ffffffffffffffffffffffffffffffff 0000000180005d70     MSVCRT:utility.obj
 0002:00001d80       _load_config_used          0000000180005d80     MSVCRT:loadcfg.obj
 0002:00001f80       _tls_used                  0000000180005f80     MSVCRT:tlssup.obj
 0002:00001fa8       __volatile_metadata        0000000180005fa8     <linker-defined>
 0002:00002370       __rtc_iaa                  0000000180006370     MSVCRT:initsect.obj
 0002:00002378       __rtc_izz                  0000000180006378     MSVCRT:initsect.obj
 0002:00002380       __rtc_taa                  0000000180006380     MSVCRT:initsect.obj
 0002:00002388       __rtc_tzz                  0000000180006388     MSVCRT:initsect.obj
 0002:00002390       _tls_start                 0000000180006390     MSVCRT:tlssup.obj
 0002:00002394       _Init_thread_epoch         0000000180006394     MSVCRT:thread_safe_statics.obj
 0002:00002398       _tls_end                   0000000180006398     MSVCRT:tlssup.obj
 0002:00002b04       __IMPORT_DESCRIPTOR_KERNEL32 0000000180006b04     kernel32:KERNEL32.dll
 0002:00002b18       __IMPORT_DESCRIPTOR_VCRUNTIME140 0000000180006b18     vcruntime:VCRUNTIME140.dll
 0002:00002b2c       __IMPORT_DESCRIPTOR_api-ms-win-crt-runtime-l1-1-0 0000000180006b2c     ucrt:api-ms-win-crt-runtime-l1-1-0.dll
 0002:00002b40       __IMPORT_DESCRIPTOR_api-ms-win-crt-stdio-l1-1-0 0000000180006b40     ucrt:api-ms-win-crt-stdio-l1-1-0.dll
 0002:00002b54       __IMPORT_DESCRIPTOR_api-ms-win-crt-string-l1-1-0 0000000180006b54     ucrt:api-ms-win-crt-string-l1-1-0.dll
 0002:00002b68       __NULL_IMPORT_DESCRIPTOR   0000000180006b68     kernel32:KERNEL32.dll
 0003:00000120       _Init_global_epoch         0000000180008120     MSVCRT:thread_safe_statics.obj
 0003:00000130       __security_cookie          0000000180008130     MSVCRT:gs_cookie.obj
 0003:00000138       __security_cookie_complement 0000000180008138     MSVCRT:gs_cookie.obj
 0003:00000140       __scrt_native_dllmain_reason 0000000180008140     MSVCRT:utility.obj
 0003:00000148       __isa_available            0000000180008148     MSVCRT:cpu_disp.obj
 0003:0000014c       __isa_enabled              000000018000814c     MSVCRT:cpu_disp.obj
 0003:00000150       __memset_fast_string_threshold 0000000180008150     MSVCRT:cpu_disp.obj
 0003:00000158       __memset_nt_threshold      0000000180008158     MSVCRT:cpu_disp.obj
 0003:00000160       __scrt_ucrt_dll_is_in_use  0000000180008160     MSVCRT:ucrt_stubs.obj
 0003:00000170       g_wrongHeapCallbacks       0000000180008170     libsetfldw001.obj
 0003:000001f0       g_szTagInfo                00000001800081f0     libsetfldw001.obj
 0003:00002130       g_tagFlags                 000000018000a130     libsetfldw001.obj
 0003:00002518       g_refsToVerifyCnt          000000018000a518     libsetfldw001.obj
 0003:0000251c       g_fakeUserData             000000018000a51c     libsetfldw001.obj
 0003:00002520       g_tagVisitCount            000000018000a520     libsetfldw001.obj
 0003:000034c0       g_refsToVerify             000000018000b4c0     libsetfldw001.obj
 0003:0001abc0       g_userDataError            0000000180022bc0     libsetfldw001.obj
 0003:0001aea8       ?_OptionsStorage@?1??__local_stdio_printf_options@@9@4_KA 0000000180022ea8     libsetfldw001.obj
 0003:0001b468       _tls_index                 0000000180023468     MSVCRT:tlssup.obj
 0003:0001b470       __scrt_current_native_startup_state 0000000180023470     MSVCRT:utility.obj
 0003:0001b478       __scrt_native_startup_lock 0000000180023478     MSVCRT:utility.obj
 0003:0001b4b8       __scrt_debugger_hook_flag  00000001800234b8     MSVCRT:utility_desktop.obj
 0003:0001b4c0       ?__type_info_root_node@@3U__type_info_node@@A 00000001800234c0     MSVCRT:tncleanup.obj
 0003:0001b4d0       ?_OptionsStorage@?1??__local_stdio_scanf_options@@9@4_KA 00000001800234d0     MSVCRT:default_local_stdio_options.obj
 0003:0001b4d8       __favor                    00000001800234d8     MSVCRT:cpu_disp.obj
 0003:0001b4e0       __dyn_tls_init_callback    00000001800234e0     <common>

 entry point at        0001:00002450

 Static symbols

 0000:fffda000       .debug$S                   0000000180000000     setfldw001.exp
 0000:fffda000       .debug$S                   0000000180000000     vcruntime:VCRUNTIME140.dll
 0000:fffda000       .debug$S                   0000000180000000     vcruntime:VCRUNTIME140.dll
 0000:fffda000       .debug$S                   0000000180000000     vcruntime:VCRUNTIME140.dll
 0000:fffda000       .debug$S                   0000000180000000     vcruntime:VCRUNTIME140.dll
 0000:fffda000       .debug$S                   0000000180000000     vcruntime:VCRUNTIME140.dll
 0000:fffda000       .debug$S                   0000000180000000     vcruntime:VCRUNTIME140.dll
 0000:fffda000       .debug$S                   0000000180000000     vcruntime:VCRUNTIME140.dll
 0000:fffda000       .debug$S                   0000000180000000     ucrt:api-ms-win-crt-convert-l1-1-0.dll
 0002:ffffc000       .idata$6                   0000000180000000     ucrt:api-ms-win-crt-convert-l1-1-0.dll
 0000:fffda000       .debug$S                   0000000180000000     ucrt:api-ms-win-crt-heap-l1-1-0.dll
 0000:fffda000       .debug$S                   0000000180000000     ucrt:api-ms-win-crt-heap-l1-1-0.dll
 0000:fffda000       .debug$S                   0000000180000000     ucrt:api-ms-win-crt-heap-l1-1-0.dll
 0000:fffda000       .debug$S                   0000000180000000     ucrt:api-ms-win-crt-heap-l1-1-0.dll
 0002:ffffc000       .idata$6                   0000000180000000     ucrt:api-ms-win-crt-heap-l1-1-0.dll
 0000:fffda000       .debug$S                   0000000180000000     ucrt:api-ms-win-crt-runtime-l1-1-0.dll
 0000:fffda000       .debug$S                   0000000180000000     ucrt:api-ms-win-crt-runtime-l1-1-0.dll
 0000:fffda000       .debug$S                   0000000180000000     ucrt:api-ms-win-crt-runtime-l1-1-0.dll
 0000:fffda000       .debug$S                   0000000180000000     ucrt:api-ms-win-crt-runtime-l1-1-0.dll
 0000:fffda000       .debug$S                   0000000180000000     ucrt:api-ms-win-crt-runtime-l1-1-0.dll
 0000:fffda000       .debug$S                   0000000180000000     ucrt:api-ms-win-crt-runtime-l1-1-0.dll
 0000:fffda000       .debug$S                   0000000180000000     ucrt:api-ms-win-crt-runtime-l1-1-0.dll
 0000:fffda000       .debug$S                   0000000180000000     ucrt:api-ms-win-crt-runtime-l1-1-0.dll
 0000:fffda000       .debug$S                   0000000180000000     ucrt:api-ms-win-crt-runtime-l1-1-0.dll
 0000:fffda000       .debug$S                   0000000180000000     ucrt:api-ms-win-crt-runtime-l1-1-0.dll
 0000:fffda000       .debug$S                   0000000180000000     ucrt:api-ms-win-crt-runtime-l1-1-0.dll
 0000:fffda000       .debug$S                   0000000180000000     ucrt:api-ms-win-crt-runtime-l1-1-0.dll
 0000:fffda000       .debug$S                   0000000180000000     ucrt:api-ms-win-crt-runtime-l1-1-0.dll
 0000:fffda000       .debug$S                   0000000180000000     ucrt:api-ms-win-crt-runtime-l1-1-0.dll
 0000:fffda000       .debug$S                   0000000180000000     ucrt:api-ms-win-crt-runtime-l1-1-0.dll
 0000:fffda000       .debug$S                   0000000180000000     ucrt:api-ms-win-crt-runtime-l1-1-0.dll
 0000:fffda000       .debug$S                   0000000180000000     ucrt:api-ms-win-crt-stdio-l1-1-0.dll
 0000:fffda000       .debug$S                   0000000180000000     ucrt:api-ms-win-crt-stdio-l1-1-0.dll
 0000:fffda000       .debug$S                   0000000180000000     ucrt:api-ms-win-crt-stdio-l1-1-0.dll
 0000:fffda000       .debug$S                   0000000180000000     ucrt:api-ms-win-crt-stdio-l1-1-0.dll
 0000:fffda000       .debug$S                   0000000180000000     ucrt:api-ms-win-crt-stdio-l1-1-0.dll
 0000:fffda000       .debug$S                   0000000180000000     ucrt:api-ms-win-crt-stdio-l1-1-0.dll
 0000:fffda000       .debug$S                   0000000180000000     ucrt:api-ms-win-crt-stdio-l1-1-0.dll
 0000:fffda000       .debug$S                   0000000180000000     ucrt:api-ms-win-crt-stdio-l1-1-0.dll
 0000:fffda000       .debug$S                   0000000180000000     ucrt:api-ms-win-crt-stdio-l1-1-0.dll
 0000:fffda000       .debug$S                   0000000180000000     ucrt:api-ms-win-crt-stdio-l1-1-0.dll
 0000:fffda000       .debug$S                   0000000180000000     ucrt:api-ms-win-crt-string-l1-1-0.dll
 0000:fffda000       .debug$S                   0000000180000000     ucrt:api-ms-win-crt-string-l1-1-0.dll
 0000:fffda000       .debug$S                   0000000180000000     ucrt:api-ms-win-crt-string-l1-1-0.dll
 0000:fffda000       .debug$S                   0000000180000000     ucrt:api-ms-win-crt-string-l1-1-0.dll
 0000:fffda000       .debug$S                   0000000180000000     ucrt:api-ms-win-crt-string-l1-1-0.dll
 0000:fffda000       .debug$S                   0000000180000000     ucrt:api-ms-win-crt-string-l1-1-0.dll
 0000:fffda000       .debug$S                   0000000180000000     ucrt:api-ms-win-crt-string-l1-1-0.dll
 0000:fffda000       .debug$S                   0000000180000000     ucrt:api-ms-win-crt-string-l1-1-0.dll
 0000:fffda000       .debug$S                   0000000180000000     ucrt:api-ms-win-crt-string-l1-1-0.dll
 0000:fffda000       .debug$S                   0000000180000000     kernel32:KERNEL32.dll
 0000:fffda000       .debug$S                   0000000180000000     kernel32:KERNEL32.dll
 0000:fffda000       .debug$S                   0000000180000000     kernel32:KERNEL32.dll
 0000:fffda000       .debug$S                   0000000180000000     kernel32:KERNEL32.dll
 0000:fffda000       .debug$S                   0000000180000000     kernel32:KERNEL32.dll
 0000:fffda000       .debug$S                   0000000180000000     kernel32:KERNEL32.dll
 0000:fffda000       .debug$S                   0000000180000000     kernel32:KERNEL32.dll
 0000:fffda000       .debug$S                   0000000180000000     kernel32:KERNEL32.dll
 0000:fffda000       .debug$S                   0000000180000000     kernel32:KERNEL32.dll
 0000:fffda000       .debug$S                   0000000180000000     kernel32:KERNEL32.dll
 0000:fffda000       .debug$S                   0000000180000000     kernel32:KERNEL32.dll
 0000:fffda000       .debug$S                   0000000180000000     kernel32:KERNEL32.dll
 0000:fffda000       .debug$S                   0000000180000000     kernel32:KERNEL32.dll
 0000:fffda000       .debug$S                   0000000180000000     kernel32:KERNEL32.dll
 0000:fffda000       .debug$S                   0000000180000000     kernel32:KERNEL32.dll
 0000:fffda000       .debug$S                   0000000180000000     kernel32:KERNEL32.dll
 0000:fffda000       .debug$S                   0000000180000000     kernel32:KERNEL32.dll
 0000:fffda000       .debug$S                   0000000180000000     kernel32:KERNEL32.dll
 0000:fffda000       .debug$S                   0000000180000000     kernel32:KERNEL32.dll
 0000:fffda000       .debug$S                   0000000180000000     kernel32:KERNEL32.dll
 0000:fffda000       .debug$S                   0000000180000000     kernel32:KERNEL32.dll
 0000:fffda000       .debug$S                   0000000180000000     kernel32:KERNEL32.dll
 0000:fffda000       .debug$S                   0000000180000000     kernel32:KERNEL32.dll
 0000:fffda000       .debug$S                   0000000180000000     kernel32:KERNEL32.dll
 0000:fffda000       .debug$S                   0000000180000000     kernel32:KERNEL32.dll
 0000:fffda000       .debug$S                   0000000180000000     kernel32:KERNEL32.dll
 0000:fffda000       .debug$S                   0000000180000000     kernel32:KERNEL32.dll
 0000:fffda000       .debug$S                   0000000180000000     kernel32:KERNEL32.dll
 0001:00000fd4       addRefToVerify             0000000180001fd4 f   libsetfldw001.obj
 0001:00001048       agentThreadWrapper         0000000180002048 f   libsetfldw001.obj
 0001:00001220       file_basename              0000000180002220 f   libsetfldw001.obj
 0001:0000195c       startAgentThreadWrapper    000000018000295c f   libsetfldw001.obj
 0001:00001c88       syncDebuggeeStatus         0000000180002c88 f   libsetfldw001.obj
 0001:00001f10       capture_previous_context   0000000180002f10 f   MSVCRT:gs_report.obj
 0001:00001f84       ?__scrt_initialize_thread_safe_statics@@YAHXZ 0000000180002f84 f   MSVCRT:thread_safe_statics.obj
 0001:00002054       ?__scrt_uninitialize_thread_safe_statics@@YAXXZ 0000000180003054 f   MSVCRT:thread_safe_statics.obj
 0001:00002100       $$000000                   0000000180003100     MSVCRT:amdsecgs.obj
 0001:00002130       ?dllmain_crt_dispatch@@YAHQEAUHINSTANCE__@@KQEAX@Z 0000000180003130 f   MSVCRT:dll_dllmain.obj
 0001:00002180       ?dllmain_crt_process_attach@@YAHQEAUHINSTANCE__@@QEAX@Z 0000000180003180 f   MSVCRT:dll_dllmain.obj
 0001:00002298       ?dllmain_crt_process_detach@@YAH_N@Z 0000000180003298 f   MSVCRT:dll_dllmain.obj
 0001:0000231c       ?dllmain_dispatch@@YAHQEAUHINSTANCE__@@KQEAX@Z 000000018000331c f   MSVCRT:dll_dllmain.obj
 0001:00002d30       $$000000                   0000000180003d30     MSVCRT:guard_dispatch.obj
 0001:00002d50       $$000000                   0000000180003d50     MSVCRT:guard_xfg_dispatch.obj
 0001:00002d66       ?fin$0@?0??dllmain_crt_process_attach@@YAHQEAUHINSTANCE__@@QEAX@Z@4HA 0000000180003d66 f   MSVCRT:dll_dllmain.obj
 0001:00002d7d       ?fin$0@?0??dllmain_crt_process_detach@@YAH_N@Z@4HA 0000000180003d7d f   MSVCRT:dll_dllmain.obj
 0001:00002d96       ?fin$1@?0??dllmain_crt_process_detach@@YAH_N@Z@4HA 0000000180003d96 f   MSVCRT:dll_dllmain.obj
 0001:00002daa       ?filt$0@?0??dllmain_dispatch@@YAHQEAUHINSTANCE__@@KQEAX@Z@4HA 0000000180003daa f   MSVCRT:dll_dllmain.obj
 0001:00002de0       __scrt_is_nonwritable_in_current_image$filt$0 0000000180003de0 f   MSVCRT:utility.obj
 0002:000001e8       ?__scrt_initialize_tss_var@@3P6AHXZEA 00000001800041e8     MSVCRT:thread_safe_statics.obj
 0002:00000310       ?opcLengths@@3QBEB         0000000180004310     libsetfldw001.obj
 0002:00001cb0       GS_ExceptionPointers       0000000180005cb0     MSVCRT:gs_report.obj
 0002:000023a0       $unwind$fprintf            00000001800063a0     libsetfldw001.obj
 0002:000023ac       $unwind$printf             00000001800063ac     libsetfldw001.obj
 0002:000023b8       $unwind$?NewObject@JNIEnv_@@QEAAPEAV_jobject@@PEAV_jclass@@PEAU_jmethodID@@ZZ 00000001800063b8     libsetfldw001.obj
 0002:000023b8       $unwind$nsk_lcomplain      00000001800063b8     libsetfldw001.obj
 0002:000023b8       $unwind$nsk_ldisplay       00000001800063b8     libsetfldw001.obj
 0002:000023c0       $unwind$Java_nsk_jvmti_SetFieldAccessWatch_setfldw001_touchfld0 00000001800063c0     libsetfldw001.obj
 0002:000023c0       $unwind$nsk_lvdisplay      00000001800063c0     libsetfldw001.obj
 0002:000023c0       $unwind$_RTC_Initialize    00000001800063c0     MSVCRT:initsect.obj
 0002:000023c0       $unwind$_RTC_Terminate     00000001800063c0     MSVCRT:initsect.obj
 0002:000023c0       $unwind$?__scrt_initialize_thread_safe_statics@@YAHXZ 00000001800063c0     MSVCRT:thread_safe_statics.obj
 0002:000023cc       $unwind$nsk_lvcomplain     00000001800063cc     libsetfldw001.obj
 0002:000023e4       $unwind$nsk_ltrace         00000001800063e4     libsetfldw001.obj
 0002:000023e4       $unwind$__report_gsfailure 00000001800063e4     MSVCRT:gs_report.obj
 0002:000023ec       $unwind$Agent_Initialize   00000001800063ec     libsetfldw001.obj
 0002:000023ec       $unwind$nsk_lvtrace        00000001800063ec     libsetfldw001.obj
 0002:000023ec       $unwind$__raise_securityfailure 00000001800063ec     MSVCRT:gs_report.obj
 0002:000023ec       $unwind$__scrt_initialize_crt 00000001800063ec     MSVCRT:utility.obj
 0002:000023ec       $unwind$__scrt_initialize_onexit_tables 00000001800063ec     MSVCRT:utility.obj
 0002:000023ec       $unwind$__scrt_release_startup_lock 00000001800063ec     MSVCRT:utility.obj
 0002:000023ec       $unwind$__scrt_uninitialize_crt 00000001800063ec     MSVCRT:utility.obj
 0002:000023ec       $unwind$_onexit            00000001800063ec     MSVCRT:utility.obj
 0002:000023f4       $unwind$nsk_lverify        00000001800063f4     libsetfldw001.obj
 0002:00002404       $unwind$nsk_vprintf        0000000180006404     libsetfldw001.obj
 0002:00002414       $unwind$nsk_printf         0000000180006414     libsetfldw001.obj
 0002:0000241c       $unwind$?nsk_jni_lverify@@YAHHPEAUJNIEnv_@@HQEBDH1ZZ 000000018000641c     libsetfldw001.obj
 0002:00002430       $unwind$?nsk_jni_check_exception@@YAHPEAUJNIEnv_@@QEBDH@Z 0000000180006430     libsetfldw001.obj
 0002:0000244c       $unwind$Java_nsk_jvmti_SetFieldAccessWatch_setfldw001_check 000000018000644c     libsetfldw001.obj
 0002:0000244c       $unwind$Java_nsk_jvmti_unit_FollowReferences_FollowRefObjects_resetTags 000000018000644c     libsetfldw001.obj
 0002:0000244c       $unwind$addRefToVerify     000000018000644c     libsetfldw001.obj
 0002:0000244c       $unwind$nsk_jvmti_resetAgentData 000000018000644c     libsetfldw001.obj
 0002:0000244c       $unwind$__scrt_initialize_default_local_stdio_options 000000018000644c     MSVCRT:default_local_stdio_options.obj
 0002:0000244c       $unwind$?dllmain_crt_dispatch@@YAHQEAUHINSTANCE__@@KQEAX@Z 000000018000644c     MSVCRT:dll_dllmain.obj
 0002:0000244c       $unwind$DllMain            000000018000644c     MSVCRT:dll_dllmain_stub.obj
 0002:0000244c       $unwind$__GSHandlerCheck   000000018000644c     MSVCRT:gshandler.obj
 0002:0000244c       $unwind$?__scrt_uninitialize_thread_safe_statics@@YAXXZ 000000018000644c     MSVCRT:thread_safe_statics.obj
 0002:0000244c       $unwind$__scrt_acquire_startup_lock 000000018000644c     MSVCRT:utility.obj
 0002:0000244c       $unwind$__scrt_dllmain_after_initialize_c 000000018000644c     MSVCRT:utility.obj
 0002:0000244c       $unwind$__scrt_dllmain_before_initialize_c 000000018000644c     MSVCRT:utility.obj
 0002:0000244c       $unwind$__scrt_dllmain_crt_thread_attach 000000018000644c     MSVCRT:utility.obj
 0002:0000244c       $unwind$__scrt_dllmain_crt_thread_detach 000000018000644c     MSVCRT:utility.obj
 0002:0000244c       $unwind$__scrt_dllmain_uninitialize_c 000000018000644c     MSVCRT:utility.obj
 0002:0000244c       $unwind$__scrt_dllmain_uninitialize_critical 000000018000644c     MSVCRT:utility.obj
 0002:0000244c       $unwind$atexit             000000018000644c     MSVCRT:utility.obj
 0002:00002454       $unwind$nsk_jvmti_lverify  0000000180006454     libsetfldw001.obj
 0002:00002468       $unwind$exitOnError        0000000180006468     libsetfldw001.obj
 0002:00002478       $unwind$Java_nsk_share_jvmti_ArgumentHandler_getAgentOptionsString 0000000180006478     libsetfldw001.obj
 0002:0000248c       $unwind$Java_nsk_jvmti_unit_FollowReferences_FollowRefObjects_getTag 000000018000648c     libsetfldw001.obj
 0002:0000248c       $unwind$Java_nsk_share_jvmti_DebugeeClass_checkStatus 000000018000648c     libsetfldw001.obj
 0002:0000248c       $unwind$agentThreadWrapper 000000018000648c     libsetfldw001.obj
 0002:0000249c       $unwind$startAgentThreadWrapper 000000018000649c     libsetfldw001.obj
 0002:000024b8       $unwind$syncDebuggeeStatus 00000001800064b8     libsetfldw001.obj
 0002:000024b8       $unwind$__scrt_dllmain_exception_filter 00000001800064b8     MSVCRT:utility.obj
 0002:000024cc       $unwind$Java_nsk_share_jvmti_DebugeeClass_resetAgentData 00000001800064cc     libsetfldw001.obj
 0002:000024d4       $unwind$MA_checkStatus     00000001800064d4     libsetfldw001.obj
 0002:000024e8       $unwind$Java_nsk_jvmti_unit_FollowReferences_FollowRefObjects_setTag 00000001800064e8     libsetfldw001.obj
 0002:00002500       $unwind$Java_nsk_jvmti_unit_FollowReferences_FollowRefObjects_addRefToVerify 0000000180006500     libsetfldw001.obj
 0002:0000251c       $unwind$setWatch           000000018000651c     libsetfldw001.obj
 0002:00002534       $unwind$FieldAccess        0000000180006534     libsetfldw001.obj
 0002:0000254c       $unwind$capture_previous_context 000000018000654c     MSVCRT:gs_report.obj
 0002:00002558       $unwind$__GSHandlerCheckCommon 0000000180006558     MSVCRT:gshandler.obj
 0002:00002560       $xdatasym                  0000000180006560     MSVCRT:amdsecgs.obj
 0002:00002564       $unwind$?dllmain_crt_process_attach@@YAHQEAUHINSTANCE__@@QEAX@Z 0000000180006564     MSVCRT:dll_dllmain.obj
 0002:000025a0       $unwind$?fin$0@?0??dllmain_crt_process_attach@@YAHQEAUHINSTANCE__@@QEAX@Z@4HA 00000001800065a0     MSVCRT:dll_dllmain.obj
 0002:000025a0       $unwind$?fin$0@?0??dllmain_crt_process_detach@@YAH_N@Z@4HA 00000001800065a0     MSVCRT:dll_dllmain.obj
 0002:000025a0       $unwind$?fin$1@?0??dllmain_crt_process_detach@@YAH_N@Z@4HA 00000001800065a0     MSVCRT:dll_dllmain.obj
 0002:000025a8       $unwind$?dllmain_crt_process_detach@@YAH_N@Z 00000001800065a8     MSVCRT:dll_dllmain.obj
 0002:000025fc       $unwind$?dllmain_dispatch@@YAHQEAUHINSTANCE__@@KQEAX@Z 00000001800065fc     MSVCRT:dll_dllmain.obj
 0002:00002624       $unwind$?filt$0@?0??dllmain_dispatch@@YAHQEAUHINSTANCE__@@KQEAX@Z@4HA 0000000180006624     MSVCRT:dll_dllmain.obj
 0002:0000262c       $unwind$_DllMainCRTStartup 000000018000662c     MSVCRT:dll_dllmain.obj
 0002:0000263c       $unwind$__scrt_is_nonwritable_in_current_image 000000018000663c     MSVCRT:utility.obj
 0002:0000265c       $unwind$__scrt_is_nonwritable_in_current_image$filt$0 000000018000665c     MSVCRT:utility.obj
 0002:00002664       $unwind$__scrt_fastfail    0000000180006664     MSVCRT:utility_desktop.obj
 0002:00002674       $unwind$__security_init_cookie 0000000180006674     MSVCRT:gs_support.obj
 0002:00002680       $unwind$__isa_available_init 0000000180006680     MSVCRT:cpu_disp.obj
 0002:00002690       $xdatasym                  0000000180006690     MSVCRT:guard_dispatch.obj
 0002:00002698       $xdatasym                  0000000180006698     MSVCRT:guard_xfg_dispatch.obj
 0002:000026a0       .edata                     00000001800066a0     setfldw001.exp
 0002:000026c8       rgpv                       00000001800066c8     setfldw001.exp
 0002:00002710       rgszName                   0000000180006710     setfldw001.exp
 0002:00002758       rgwOrd                     0000000180006758     setfldw001.exp
 0002:0000277c       szName                     000000018000677c     setfldw001.exp
 0002:0000278b       $N00001                    000000018000678b     setfldw001.exp
 0002:0000279a       $N00002                    000000018000679a     setfldw001.exp
 0002:000027a7       $N00003                    00000001800067a7     setfldw001.exp
 0002:000027db       $N00004                    00000001800067db     setfldw001.exp
 0002:00002810       $N00005                    0000000180006810     setfldw001.exp
 0002:00002847       $N00006                    0000000180006847     setfldw001.exp
 0002:0000287f       $N00007                    000000018000687f     setfldw001.exp
 0002:000028c4       $N00008                    00000001800068c4     setfldw001.exp
 0002:00002901       $N00009                    0000000180006901     setfldw001.exp
 0002:00002949       $N00010                    0000000180006949     setfldw001.exp
 0002:00002989       $N00011                    0000000180006989     setfldw001.exp
 0002:000029c6       $N00012                    00000001800069c6     setfldw001.exp
 0002:00002a01       $N00013                    0000000180006a01     setfldw001.exp
 0002:00002a2f       $N00014                    0000000180006a2f     setfldw001.exp
 0002:00002a60       $N00015                    0000000180006a60     setfldw001.exp
 0002:00002a8f       $N00016                    0000000180006a8f     setfldw001.exp
 0002:00002abe       $N00017                    0000000180006abe     setfldw001.exp
 0002:00002af3       $N00018                    0000000180006af3     setfldw001.exp
 0002:00002f02       .idata$6                   0000000180006f02     kernel32:KERNEL32.dll
 0002:00002f66       .idata$6                   0000000180006f66     vcruntime:VCRUNTIME140.dll
 0002:000030d2       .idata$6                   00000001800070d2     ucrt:api-ms-win-crt-runtime-l1-1-0.dll
 0002:000030f4       .idata$6                   00000001800070f4     ucrt:api-ms-win-crt-stdio-l1-1-0.dll
 0002:00003114       .idata$6                   0000000180007114     ucrt:api-ms-win-crt-string-l1-1-0.dll
 0003:00000000       ?codeAttributeName@@3PEBDEB 0000000180008000     libsetfldw001.obj
 0003:00000008       ?lineNumberAttributeName@@3PEBDEB 0000000180008008     libsetfldw001.obj
 0003:00000010       ?localVarAttributeName@@3PEBDEB 0000000180008010     libsetfldw001.obj
 0003:00000018       ?localVarTypeAttributeName@@3PEBDEB 0000000180008018     libsetfldw001.obj
 0003:00000020       ?stackMapAttributeName@@3PEBDEB 0000000180008020     libsetfldw001.obj
 0003:00000028       ?callBytes@@3PAEA          0000000180008028     libsetfldw001.obj
 0003:0000002c       ?allocBytes@@3PAEA         000000018000802c     libsetfldw001.obj
 0003:00000030       fields                     0000000180008030     libsetfldw001.obj
 0003:0001abc4       redefineAttempted          0000000180022bc4     libsetfldw001.obj
 0003:0001abc8       nsk_context                0000000180022bc8     libsetfldw001.obj
 0003:0001abd4       redefineSucceed            0000000180022bd4     libsetfldw001.obj
 0003:0001abd8       agentFailed                0000000180022bd8     libsetfldw001.obj
 0003:0001abdc       currentAgentStatus         0000000180022bdc     libsetfldw001.obj
 0003:0001abe0       context                    0000000180022be0     libsetfldw001.obj
 0003:0001ac98       agentThread                0000000180022c98     libsetfldw001.obj
 0003:0001aca0       agentThreadProc            0000000180022ca0     libsetfldw001.obj
 0003:0001aca8       agentThreadArg             0000000180022ca8     libsetfldw001.obj
 0003:0001acb0       agent_data                 0000000180022cb0     libsetfldw001.obj
 0003:0001acc0       jvmti_env                  0000000180022cc0     libsetfldw001.obj
 0003:0001acc8       jvm                        0000000180022cc8     libsetfldw001.obj
 0003:0001acd0       jni_env                    0000000180022cd0     libsetfldw001.obj
 0003:0001acd8       checkStatus_func           0000000180022cd8     libsetfldw001.obj
 0003:0001ace0       ?codeAttributeIndex@@3GA   0000000180022ce0     libsetfldw001.obj
 0003:0001ace4       ?lineNumberAttributeIndex@@3GA 0000000180022ce4     libsetfldw001.obj
 0003:0001ace8       ?localVarAttributeIndex@@3GA 0000000180022ce8     libsetfldw001.obj
 0003:0001acec       ?localVarTypeAttributeIndex@@3GA 0000000180022cec     libsetfldw001.obj
 0003:0001acf0       ?stackMapAttributeIndex@@3GA 0000000180022cf0     libsetfldw001.obj
 0003:0001acf4       ?stackFrameOffset@@3GA     0000000180022cf4     libsetfldw001.obj
 0003:0001acf8       ?mode@@3HA                 0000000180022cf8     libsetfldw001.obj
 0003:0001acfc       ?constantPoolSize@@3GA     0000000180022cfc     libsetfldw001.obj
 0003:0001ad00       ?orig@@3PEBEEB             0000000180022d00     libsetfldw001.obj
 0003:0001ad08       ?gen@@3PEAEEA              0000000180022d08     libsetfldw001.obj
 0003:0001ad10       ?inputPos@@3PEAEEA         0000000180022d10     libsetfldw001.obj
 0003:0001ad18       ?endPos@@3PEBEEB           0000000180022d18     libsetfldw001.obj
 0003:0001ad20       ?genPos@@3PEAEEA           0000000180022d20     libsetfldw001.obj
 0003:0001ad28       ?markPos@@3PEAEEA          0000000180022d28     libsetfldw001.obj
 0003:0001ad30       ?constantPool@@3PEAPEADEA  0000000180022d30     libsetfldw001.obj
 0003:0001ad38       ?constantPoolCount@@3GA    0000000180022d38     libsetfldw001.obj
 0003:0001ad3c       ?zeroBytes@@3PAEA          0000000180022d3c     libsetfldw001.obj
 0003:0001ad40       ?codeLength@@3IA           0000000180022d40     libsetfldw001.obj
 0003:0001ad44       result                     0000000180022d44     libsetfldw001.obj
 0003:0001ad48       ?map@@3PEAIEA              0000000180022d48     libsetfldw001.obj
 0003:0001ad50       ?widening@@3PEACEA         0000000180022d50     libsetfldw001.obj
 0003:0001ad58       jvmti                      0000000180022d58     libsetfldw001.obj
 0003:0001ad60       callbacks                  0000000180022d60     libsetfldw001.obj
 0003:0001ae98       caps                       0000000180022e98     libsetfldw001.obj
 0003:0001aeb0       GS_ExceptionRecord         0000000180022eb0     MSVCRT:gs_report.obj
 0003:0001af50       GS_ContextRecord           0000000180022f50     MSVCRT:gs_report.obj
 0003:0001b420       ?g_tss_cv@@3U_RTL_CONDITION_VARIABLE@@A 0000000180023420     MSVCRT:thread_safe_statics.obj
 0003:0001b428       ?g_tss_event@@3PEAXEA      0000000180023428     MSVCRT:thread_safe_statics.obj
 0003:0001b430       ?g_tss_mutex@@3U_RTL_CRITICAL_SECTION@@A 0000000180023430     MSVCRT:thread_safe_statics.obj
 0003:0001b458       ?g_sleep_condition_variable_cs@@3P6AHPEAU_RTL_CONDITION_VARIABLE@@PEAU_RTL_CRITICAL_SECTION@@K@ZEA 0000000180023458     MSVCRT:thread_safe_statics.obj
 0003:0001b460       ?g_wake_all_condition_variable@@3P6AXPEAU_RTL_CONDITION_VARIABLE@@@ZEA 0000000180023460     MSVCRT:thread_safe_statics.obj
 0003:0001b46c       ?__proc_attached@@3HA      000000018002346c     MSVCRT:dll_dllmain.obj
 0003:0001b480       ?is_initialized_as_dll@@3_NA 0000000180023480     MSVCRT:utility.obj
 0003:0001b481       ?module_local_atexit_table_initialized@@3_NA 0000000180023481     MSVCRT:utility.obj
 0003:0001b488       ?module_local_atexit_table@@3U_onexit_table_t@@A 0000000180023488     MSVCRT:utility.obj
 0003:0001b4a0       ?module_local_at_quick_exit_table@@3U_onexit_table_t@@A 00000001800234a0     MSVCRT:utility.obj
